:020000040000fa
:080000000002040000000000f2
:020000040000fa
:10000800d8020000d8020000d8020000d802000080
:10001800d8020000d8020000d8020000d802000070
:10002800d8020000d8020000d8020000d802000060
:10003800d8020000d8020000d802000048310000b1
:10004800d8020000d8020000d80200001e280000d4
:10005800e0270000d8020000d8020000d802000003
:10006800d8020000d8020000d8020000d802000020
:10007800d8020000d8020000d8020000d802000010
:10008800d8020000d8020000d8020000d802000000
:10009800d8020000d80200009c2800005e2800005a
:1000a800d8020000d8020000d8020000d8020000e0
:1000b800d8020000d8020000d8020000d8020000d0
:1000c800d8020000d8020000d8020000d8020000c0
:1000d800d8020000d8020000d8020000d8020000b0
:1000e800d8020000d8020000d8020000d8020000a0
:1000f800d8020000d8020000d8020000d802000090
:10010800d8020000d8020000d8020000d80200007f
:10011800d8020000d8020000d8020000d80200006f
:10012800d8020000d8020000d8020000d80200005f
:10013800d8020000d8020000d8020000d80200004f
:10014800d8020000d8020000d8020000d80200003f
:10015800d8020000d8020000d8020000d80200002f
:10016800d8020000d80200001a290000dc2800008c
:10017800d8020000d8020000d8020000d80200000f
:10018800d8020000d8020000d8020000d8020000ff
:10019800d8020000d8020000d8020000d8020000ef
:1001a800d8020000d8020000d8020000d8020000df
:1001b800d8020000d8020000d8020000d8020000cf
:1001c800d8020000d8020000d8020000d8020000bf
:1001d800d8020000d8020000d8020000d8020000af
:1001e800d8020000d8020000d8020000d80200009f
:0801f800d8020000d80200004b
:020000040000fa
:10020800d8020000d8020000d8020000d80200007e
:10021800d8020000d8020000d8020000d80200006e
:10022800d8020000d8020000d8020000d80200005e
:10023800d8020000d8020000d802000048310000af
:10024800d8020000d8020000d80200001e280000d2
:10025800e0270000d8020000d8020000d802000001
:10026800d8020000d8020000d8020000d80200001e
:10027800d8020000d8020000d8020000d80200000e
:10028800d8020000d8020000d8020000d8020000fe
:10029800d8020000d80200009c2800005e28000058
:1002a800d8020000d8020000d8020000d8020000de
:1002b800d8020000d8020000d8020000d8020000ce
:1002c800d8020000d8020000d8020000d8020000be
:1002d800d8020000d8020000d8020000d8020000ae
:1002e800d8020000d8020000d8020000d80200009e
:1002f800d8020000d8020000d8020000d80200008e
:10030800d8020000d8020000d8020000d80200007d
:10031800d8020000d8020000d8020000d80200006d
:10032800d8020000d8020000d8020000d80200005d
:10033800d8020000d8020000d8020000d80200004d
:10034800d8020000d8020000d8020000d80200003d
:10035800d8020000d8020000d8020000d80200002d
:10036800d8020000d80200001a290000dc2800008a
:10037800d8020000d8020000d8020000d80200000d
:10038800d8020000d8020000d8020000d8020000fd
:10039800d8020000d8020000d8020000d8020000ed
:1003a800d8020000d8020000d8020000d8020000dd
:1003b800d8020000d8020000d8020000d8020000cd
:1003c800d8020000d8020000d8020000d8020000bd
:1003d800d8020000d8020000d8020000d8020000ad
:1003e800d8020000d8020000d8020000d80200009d
:0803f800d8020000d802000049
:020000040000fa
:10040000cfbf20000e7f24000e01880000000000f6
:1004100000012000200288000c00070000322300a9
:100420000100200011000700000020000000e00093
:100430000200320000000200000000008a2d0200cd
:10044000000000000040da000000fe004440a90067
:10045000603a20000000e0000300320000002000ad
:10046000a00188004440a800000006009101880017
:10047000800078000000eb0015003700e2804000ab
:1004800032a0b4009101ba00e280400032a0b40072
:100490009102ba00e280400032a0b4000002eb00fa
:1004a000472bde00f507b200602ce10004003a00a3
:1004b0000059eb008301e900fdff3e000400370016
:1004c0006128e100010032000082eb000400070017
:1004d0001101ba000200e000e8ff3a000000060047
:1004e0003159ba008301e9000c0032002159ba00e9
:1004f0008301e900080032000400e00003003a0034
:10050000e280400032a0b400f5ff370011d9ba00f4
:100510008301e900faff3a008100e800e180400031
:1005200032a0b400000006005a29040000000000b8
:100530006e29040000000000822904000000000071
:100540009629040000000000a82904000000000013
:10055000e629040000000000242a04000000000036
:10056000642b040000000000122d040000000000b5
:100570004e2d040000000000642a0400000000006a
:100580007e2a040000000000ca2b040000000000c6
:10059000662c0400000000001a2b0400000000007c
:1005a000322b0400000000004a2b04000000000071
:1005b0000040da000000fe000003b1000b0035002f
:1005c0009000b100080034008000b1000700350041
:1005d0009001b100040034007000b1000300350048
:1005e0009001b10001003c00100005000000050072
:1005f0001004b100070035009001b1000400340080
:100600007000b100030035009001b10001003c0012
:1006100010000500000005006900e100040035003d
:100620006d00e100030034000002b100010032005f
:1006300000000500100005001004b10003003500a3
:100640009001b10001003c00100005000000050011
:10065000800078001104b100030035009101b10061
:1006600001003c000050a00000000600800078005f
:100670001106b100030035009101b10001003c00fa
:100680000050a1000000060006c2b300000278007e
:1006900004007800b042780086cf5200fbff3200a1
:1006a000e9cf5200f9ff3200d6c2b30086cf520024
:1006b00003003a000002780016c0b30005003700be
:1006c0000043eb00b7c2b30087cf520001003a00ed
:1006d000000278000000eb00020037006a00b90059
:1006e00000804200b402fb000503b100e98f520014
:1006f000faff3600e04f5300010032000000ea002c
:10070000000006000002780002003700315a78002d
:100710000201e900e00f5100fcff3a000000060072
:100720000002780084027800050278000043eb00a4
:10073000b44f1300fbff3a0031427800845a78002e
:10074000e04f5200fcff3a00000006000002780073
:100750008042eb00b4cf1200fdff3a000080ea00b7
:1007600000004200000006000c00fa00a0bf9f003d
:10077000c0bf9f00f5ff0700b0bf9f00f0bf9f0004
:10078000140c2000d4bf9f0074815700efb0970075
:100790006c805700340007000080fa00000006005b
:1007a000881f7800c05f80001905070000047800ea
:1007b0000800780098ff0700e00f5000f9ff3a00aa
:1007c000e10f440003003200c15f800008007800a0
:1007d000d40507004f04780000000600889fbe0083
:1007e0008a1f7800000478008144780002057800b0
:1007f00004fd2f0008024200e90f520002003e00f3
:10080000040478000f003700080078008aff070012
:10081000e00f500005003200e00f550003003200e9
:10082000080078008aff07000004780008007800bc
:100830006fff070000c2eb00e00f5000060032001f
:100840007805b1008984fb0000c2eb00890f5400d9
:1008500001003d0008427800044078004f05780010
:100860004f04be0000000600f0874700889fbe00ce
:100870008a9fbe008c9fbe008e1f780081bf9f00a4
:10088000f2b79f00c05f88000002eb00d4b79f0062
:10089000044478003d0137008fba97008502e800d4
:1008a00085bf9f008985fb000b0078005aff070079
:1008b000e00f500002003200b9ff0700330137009b
:1008c00054c2b30084cf540024013a00804478001d
:1008d00025c0b300004578000fb8970005467800a2
:1008e00080057800040037004cc0b30001003700d9
:1008f0002cc0b3000b0078003b42780085c6b300e3
:10090000854f5200faff320015003e00f0c252003f
:10091000854f52002e0032000a003e00ecc2520009
:10092000854f5200260032007b003e00e04f52000f
:10093000ab003200a5c2b300854f520076003a00ea
:100940001d00370035c6b300854f52005b003200f2
:100950008542e800854f52006f003a008200370060
:1009600035c7b300854f52001f00320007003e001c
:10097000e7c25200854f520011003200e3c242002c
:10098000854f520064003a007b00370055c7b30022
:10099000854f520074003200e3c24200854f52007e
:1009a0005d003a009cef9f008bbf9f000002eb00b0
:1009b000d4b79f000a0037000a45e800cdff370092
:1009c000e24f5600c8ff32008cc0b300c9ff3700a9
:1009d0009cef9f008bbf9f0015002000d5b79f00a4
:1009e0000ec1b300670037008bbf9f006cff07008c
:1009f000e04f550004003a007fb29700c40278002f
:100a0000f4b79f00e5b79f00c05f80008004070037
:100a100080057800e18f450014003a000b00780053
:100a2000d70037008fba97001502fb00848f55005e
:100a300005003a000c027800e4b79f008502e80048
:100a400085bf9f0017003700e04f550001003a00b6
:100a50000b5e78008944e9000d003200c05f800021
:100a60006b04070080057800010037006fb697001f
:100a70000b02e800e10f5200080036000b0078007e
:100a8000e5fe0700e00f5000e6ff320003003700ec
:100a90000c027800e4b79f00020037008c02780057
:100aa000e5b79f00e04f5500b8003a000844e80061
:100ab0006fb297000a4a7800b40037008bbf9f00de
:100ac000e04f550006003a000844e800ffb29700e6
:100ad00045027800f5b79f008405780001003700d3
:100ae000efb59700c05f800049040700e10f4000a8
:100af000a3003200e04f550001003a00805d78000d
:100b00008944e9004240a900f6ff3c008b027800ce
:100b1000e5b79f009d0037008484fb0004fd2f0093
:100b200009024200e90f520009003e00d6fe07000c
:100b3000804478000b02780084057800b402fb0042
:100b40000503b100e98f5200fbff360069ff370053
:100b50008bbf9f00c05f80002d040700808f540072
:100b600082003a00890037009cef9f008bbf9f00f6
:100b7000aec0b300030037009cef9f008bbf9f0007
:100b80008ec0b30006ff0700c05f8000200407008e
:100b9000800578000042eb0084ef9f00d402200023
:100ba000848f550005003a00c05f800018040700dc
:100bb0008005780015c0b30085ef9f005fb19700f6
:100bc0008e4078000b00780004ff0700e14f4000e2
:100bd0000b003a00c15f80000b007800d1040700d1
:100be000e04f54006d003a00c45f80003400900074
:100bf000700060006a0032000080eb00680037007f
:100c000004032000848f550017003a00c05f800065
:100c1000ff0307008005780084072000848f5500bb
:100c200004003a005fb29700e00f52000700320064
:100c30000a00370084052000848f550007003a0021
:100c4000dfb29700e08f520004003200c05f8000e6
:100c5000ef0307008005780003003700c15f8000c4
:100c60000b007800af0407006066b8000e82fb003e
:100c700005002000a4b79f00b5b79f002fb19700d3
:100c8000bfb197000c00be00a60507000006be001d
:100c90005fb197008e4078000b007800cffe070010
:100ca0000080fb00010020000006460081864e0007
:100cb0008944e90009003200c05f8000d4030700c6
:100cc000800578005fb197008e4078000b007800b7
:100cd000c2fe0700e14f4000e8ff3a005fb1970015
:100ce0008e4078000b007800bcfe0700e14f40000a
:100cf00003003a00c15f80000b0078008904070000
:100d00008fea9700e0cf5200020032006006160022
:100d1000e0861e00e04f55001c003a000844e80041
:100d2000ffb297000582e9009fea9700e4cf5200e6
:100d300005003a00f4b79f0084027800150278009d
:100d40000c8abe0011003700f4b79f0084027800bf
:100d5000150278000c0a78000c003700c05f800094
:100d6000ab030700808f550008003200e10f400000
:100d700003003200c15f80006a04070007003700eb
:100d8000e04f540005003a00050037000fba970005
:100d900094447800e0cf5400bffe3a000880fb0086
:100da0004f0778004f06be004f05be004f04be003f
:100db0000f01b100000006000c00fa00889fbe0081
:100dc00000047800f4ff2700d4bf9f008004eb00ec
:100dd00099bf9f0088bf9f00a8bf9f00240c2000e0
:100de000b4bf9f0078815700cfb097007080570044
:100df000070007000fba9700094a78000fba97005a
:100e0000080052004f04be000080fa0000000600f7
:100e1000ef03b000889fbe008a9fbe008c9fbe007b
:100e20008e1f780080067800d1af9f00a2b79f0088
:100e30000007eb006a033700dfa897008100e80095
:100e4000d1af9f0054c2b300844f500006003a0057
:100e5000010278000006eb0001c3b30000c2b3003a
:100e6000b7c2b3000e0037003d0290000404b20088
:100e7000040032001d027800004a7800840ee80069
:100e8000050037000000fb008d007800e10307003b
:100e9000e10f4000520332000e07e8005003370014
:100ea0008402780034437800d2c2b300824f5300ea
:100eb0000900320005003c00804f5300080032005a
:100ec000874f53000c003a0007003700814f530052
:100ed00009003a00060037000c30a000f0ff370090
:100ee0000c00a000eeff37000c10a000ecff370054
:100ef0000c20a000eaff3700620266000100320009
:100f00000c00a10068026600010032000c20a10064
:100f10000602fb000403b100e90f52000c003e0082
:100f2000050378000002eb006a22b900b603fb005b
:100f30000703b10004824300860278009603fb0099
:100f40000703b100e98f5300f7ff360008003700b0
:100f50000002eb00a7c2b300874f530004003a0021
:100f6000afb1970043027800a3b79f008502e80065
:100f70000003eb0096b79f00e6c2b300954f130045
:100f80000c003a000ce0a00064435300d54f13005e
:100f900003003200050378000000eb000900370071
:100fa000afb3970047047800a7b79f0098b79f009a
:100fb0008502e80005037800090037006a00b900df
:100fc0000080430086027800b603fb000703b100ef
:100fd000e98f5300f9ff360090b79f00f5ff370007
:100fe000b6427800d6af9f00cac6b3008acf52007f
:100ff000250032000f003c0036c6b30086cf5200f9
:101000009c00320004003c00e0cf5200f9023200a4
:101010006b4353000f00370046c6b30086cf520023
:10102000170032006543430086cf5200af003a00fc
:101030001300370036c7b30086cf52001f003200be
:1010400007003c006443530086cf52001400320076
:101050000643e80086cf5200a4003a001300370090
:1010600056c7b30086cf5200a70032006343430047
:1010700086cf52009d003a00e5779f000d003700b3
:10108000e5779f00a2003700f0036600050120000d
:10109000010032000500280005067600d0ff370069
:1010a000e5779f000c60a00099003700e5779f006e
:1010b0000c50a0000c70a00095003700e5779f0051
:1010c000afb59700cb027800abb79f00b5b79f00d4
:1010d000e08f520002003a0041bc2000b1b79f00ef
:1010e0003fb397008002eb00010037008502e80063
:1010f000e6c37a00e0cf5300fcff3a00c5b79f007b
:101100001fb19700e00f510005003200cfb19700ea
:10111000830f51000200310082027800c5b79f00a2
:10112000cfb297000004eb00850f5200010036009b
:10113000050452006806660009c2b3000f003200c1
:10114000290037003d0290000404b2000400320080
:101150001d027800094a7800840ee8000500370077
:101160008d007800000220002a030700e10f4000f4
:10117000010032000e07e8000804e900e00f540007
:10118000f0ff3a000084eb0017003700bd0290002a
:101190000504b200090032009d037800880278003f
:1011a00035437800864b7800870ee8000504780008
:1011b000e04f53000a003a00100037008802780020
:1011c0003500fb00050478008d00780084bf9f0087
:1011d000100307000fba9700e10f4000070032002c
:1011e0000e07e80005003700080278003fb49700ba
:1011f000cfb497005fb59700efb5970089027800ec
:101200008504e900e08f5200e0ff3a00b8b79f0084
:10121000c9b79f00dab79f00ebb79f0004047800be
:1012200009c2b300e00f56000f003a006c0237000d
:101230003d0290000404b200040032001d02780058
:10124000094a7800840ee800050037008d00780018
:1012500000022000ef020700e10f40000100320011
:101260000e07e8000804e900e00f5400f0ff3a0020
:101270005b023700afb0970041047800a1b79f0030
:10128000cfc4de00090578008a0578000800be009a
:101290000a01be004800de00c80add0000807200be
:1012a000e0779f007003660009003200e04f5000b5
:1012b00007003200e14f400005003200f0779f0048
:1012c000887f9f0026002000c6b79f0003003700dc
:1012d000f8779f0017002000c7b79f0078fb2f000a
:1012e00008844700b8b79f0085ff3700e5779f0067
:1012f00069fb2f0089844700b9b79f001a002000be
:10130000cab79f007eff3700e5779f000c0cb30043
:101310008c027800050cb2003b003a00e00f56004a
:1013200005003d00afb297004501be004500be007c
:10133000a5b79f000f003700f002660012003200d0
:101340002fb497004803be00a8b79f00f69f9f00e8
:1013500087a79f0098029000cfaade0095a79f0064
:10136000a5a79f007f9897008fa097001fa19700c7
:10137000afa19700b0b79f00c1b79f00d2b79f0041
:10138000e3b79f000b003700afb09700c1027800b1
:10139000a1b79f0005047800cfc4de0009057800de
:1013a0008a057800b8b79f00c9b79f00dab79f00d9
:1013b000ebb79f003fb09700cfb097005fb19700a9
:1013c000efb19700e00f5000e08f5800e00f590098
:1013d000e08f590032003d003c00b3006000b800cf
:1013e0006011b8003fb49700cfb497005fb5970085
:1013f000efb5970008045000898458000a05590089
:101400008b85590022003700e00f560005003d0093
:10141000afb297004501be004500be00a5b79f00d2
:101420000f003700f0026600120032002fb4970060
:101430004803be00a8b79f0096af9f00a7af9f00cc
:101440008004eb00b9af9f000005eb00caaf9f001e
:101450001fa89700afa897003fa99700cfa99700b2
:10146000b0b79f00c1b79f00d2b79f00e3b79f00fe
:101470000b003700afb09700c1027800a1b79f0002
:1014800005047800090020000a0020000b0020005d
:10149000b8b79f00c9b79f00dab79f00ebb79f00ae
:1014a0009fb49700e08f54000d003a001a0020000e
:1014b0009ab79f003fb09700cfb097005fb19700f9
:1014c000efb19700e00f5000e08f5800e00f590097
:1014d000e08f5900020032008000eb0091b79f00be
:1014e0000c017800020cb20082b79f0005042000b6
:1014f000850f51003400320003003c00e00f510022
:101500000800320048003700050820008fb197001e
:10151000858f510014003200050c2000858f51008a
:1015200041003a00a6b0200015c0b3003600be004e
:101530003601be003fb49700cfb497005fb5970067
:10154000efb597000040e10001c8e10002d0e100e2
:1015500003d8e100330039008542e800f4cf52009f
:10156000f2ff3a002f00370015c0b3000001200041
:10157000010020006011b8003fb49700cfb497007d
:101580005fb59700efb597000040e10001c8e100aa
:1015900002d0e10003d8e100220039004900200018
:1015a0000000d0008180d2000281d2008381d2006d
:1015b0008904e900faff3a008542e800f0cf5200c2
:1015c000edff3a001700370015c0b300800020007f
:1015d000010020006011b8003fb49700cfb497001d
:1015e0005fb59700efb597000040e10001c8e1004a
:1015f00002d0e10003d8e1000a00390039002000e0
:101600000000d0008180d2000281d2008381d2000c
:101610008904e900faff3a008542e800f5cf52005c
:10162000edff3a00e5779f006f7597008a02fb0097
:101630009fb597008b8f520002003d00eb779f0013
:10164000040037001fb09700850f500001003d00d7
:1016500095b79f00e00f520003003200e3026600de
:10166000010032000402e900050024008502660042
:10167000060032009fb09700810f52000200340034
:1016800001025200010037000002eb006f71970069
:101690008202fb008001eb00f3af9f00850f520038
:1016a0000200340085025200f5af9f00640266001c
:1016b0003b003200e202660061026600e08f5200e9
:1016c00011003200bd0290000504b2000800320093
:1016d0009d027800b6c2b300e00f52000100320054
:1016e00006c3e800864a7800850ee800150037003a
:1016f000b0022000e00f5200010032000080e8003c
:101700008d0078000c003700e00f52000e00320010
:101710003d0290000404b200050032001d02780072
:1017200005c2b300054a7800840ee80005003700c2
:101730008d00780000022000b6010700e10f400094
:10174000010032000e07e8007faa9700e00f520068
:101750004f00320008c3b300840478003d029000bb
:101760000404b200040032001d027800084a780028
:10177000840ee800050037008d007800000320008b
:10178000a4010700e10f4000010032000e07e8004d
:101790008904e900f1ff3a00f9af9f003c003700ef
:1017a000ffaa9700e08f5200140032006802660022
:1017b00012003a0008c2b300850478003d02900090
:1017c0000404b200040032001d027800084a7800c8
:1017d000840ee800050037008d007800000220002c
:1017e0008c010700e10f4000010032000e07e80005
:1017f0008904e900f1ff3a00f9af9f00e2026600b8
:1018000061026600e08f520011003200bd029000bc
:101810000504b200080032009d027800b6c2b30091
:10182000e00f52000100320006c3e800864a78004b
:10183000850ee80015003700b0022000e00f5200ce
:10184000010032000080e8008d0078000c003700b5
:10185000e00f52000e0032003d0290000404b2007e
:10186000050032001d02780005c2b300054a780069
:10187000840ee800050037008d007800000220008b
:1018800064010700e10f4000010032000e07e8008c
:101890001fb397000602e900c223dd00c7a79f001f
:1018a0006323b90006047800b8a79f004322dd0037
:1018b00025b0200085024200e5af9f00f0046600dd
:1018c000e99f9f000c0578000a02b200da9f9f0092
:1018d000aa0037009fb597008b05e9009bb79f00d2
:1018e0000fb0970001042000810f50007a003200f1
:1018f00003003c00e00f5000080032008500370074
:10190000040820000fb19700840f51005d003200e1
:10191000040c2000840f51007e003a00e00f5600b6
:101920001f003d00efa997003304be002305be0051
:101930000802be000a03be003fb09700cfb0970078
:101940005fb19700efb1970027030700e0779f0092
:101950000000fb00cf80de000101780082017800ea
:101960000802be000a03be00880307003fb29700ca
:10197000cfb297005fb39700efb397000002520019
:1019800081825a0002035b0083835b00b4b79f002f
:10199000c5b79f00d6b79f00e7b79f003500370057
:1019a000ef9a9700e08f5200220032003fb297007a
:1019b000cfb297006fab97003604be002605be007d
:1019c0000801be000400be0084bf9f00f5b79f0061
:1019d00044020700e0779f000000fb00cf80de009c
:1019e0000801be004f0207000fba9700ffb2970030
:1019f0000004520081845a00d8a79f00e9a79f00e5
:101a00008004eb00f9a79f000005eb008aaf9f0060
:101a10005fa09700efa097007fa197008fa9970084
:101a2000b0b79f00c1b79f00d2b79f00e3b79f0038
:101a300010003700efa89700110278003fb197001f
:101a400080027800811f7800110009000481d8000d
:101a50008002fd00cf007800a4002000809fbe001f
:101a6000110009008482d800010278004f00be00f6
:101a7000e4779f00ef7197000343b000e3779f0086
:101a80002400370034bb2000df9a9700e08f52001b
:101a90000100320024ba20003fb09700cfb0970079
:101aa0005fb19700efb197004fa397000603e900dd
:101ab000050033008301d1000281d3008180d3006f
:101ac0000080d300f9ff37006f00600064407800a9
:101ad000e0779f000f0037003fb29700cfb297002a
:101ae0005fb39700efb397003fa497000804e900a5
:101af000050033008703d1000683d3008582d3001d
:101b00000482d300f9ff3700674262000443b0004b
:101b1000e4779f003d0290000404b2000700320009
:101b20009d0278006f729700844a7800850ee80065
:101b3000e04f520007003a0007003700ef749700ab
:101b40000900fb008d007800b2000700e10f4000a3
:101b5000010032000e07e8004fa59700640555000c
:101b6000caa79f00bfa59700e3855500bba79f00ac
:101b70006fa8970068005000e0af9f009fb09700eb
:101b8000e08f500053ff3a006806660014003200f0
:101b90007fa99700e00f51001100340008c2b30084
:101ba000820478003d0290000404b2000400320078
:101bb0001d027800084a7800840ee800050037000e
:101bc0008d0078000002200092000700e10f400025
:101bd000010032000e07e8008904e900f1ff3a0035
:101be000dfa9970013407800e0779f00e04f500096
:101bf00091fc3a000e0078004f0778004f06be00b7
:101c00004f05be004f04be00ef03b1000000060008
:101c1000881f78000004780038029000f10262000a
:101c2000e18f520006003a00840278000520b200dd
:101c30000800320098029000e08f52000500320048
:101c4000380290000440a000340498000080eb00ab
:101c5000200037000490a10034049800180290007e
:101c6000e00f5200070034000402e9001404980059
:101c700018027800944278000580fb00040ce8000c
:101c800005003700380290000404b200ecff3a006f
:101c90000800780011000700380290000408b20024
:101ca0000c003a00fa0f500008003a002802900099
:101cb000e00f5200e2ff3200180290000402e80038
:101cc00014049800180ce900ddff3700ed0f5000f8
:101cd000e2ff32004f047800000006000200fa0024
:101ce000889fbe008a9fbe00000478000002eb00bf
:101cf0001404980038029000610262000080eb003a
:101d00004000320024bf20008042eb0094cf12003c
:101d10000f0032000bbf2000c9fd2f008b84440050
:101d20002a102000390290002410b2008a0f5200bd
:101d300002003a000900780096000700ec84440095
:101d40008b8f5400f7ff3a0024bf2000004aeb00bd
:101d500058019000e00f51000e003a001204980064
:101d600012002000ea80570048009000f7000700aa
:101d7000e10f500003003a006ff297000480fb006f
:101d800020003700380290000440a000340498007e
:101d900013003700a800900048009000eb000700f7
:101da00010049800e00f500003003200e10f4000e3
:101db0000d003a0003003700380290000440a000f4
:101dc00002003700380290000403b3003404980086
:101dd000a8029000050c78000002eb0014049800a3
:101de0000080eb000700370028029000040c780008
:101df0000000e90010049800944278000580fb0080
:101e0000040ce8004f05be004f04be000080fa003d
:101e100000000600889fbe00010478003802900090
:101e2000e20262008084eb003b0032000403780091
:101e30000620b2009802900002003a00e08f5200a3
:101e400035003a000490a000340498008004780023
:101e5000f90fb200e08f520002003a00a802900091
:101e6000050c7800ea8f540005003a000408b2001f
:101e700003003a0088007800d0002000e5ff07004a
:101e800018029000d8029000850f52000b0032001b
:101e90000402e8001404980018027800094a780047
:101ea000040ce80015c0b30024bf2000054a7800e8
:101eb000ea8f540018003a000500370088007800c7
:101ec000094078005d0007008004780012003700a8
:101ed000380290000410b2000f0032001801900088
:101ee000a800900048009000ce0007001802900063
:101ef000840f500004003200380290000403b30045
:101f0000340498008084eb000002eb001404980075
:101f100028029000040c7800090078004f04be00ed
:101f200000000600e10f400019003200310290006d
:101f30001420b200e10f520012003a002103900079
:101f4000e00f53000f00320011029000d102900008
:101f5000850f52000d00320091027800868f5200ea
:101f600002003a008508e800020037000402e80099
:101f7000940098001102e90084087800004a780073
:101f8000000006000080eb00000006000080eb006f
:101f900000000600881f78000004780038009000d8
:101fa000000278001420b200e10f520005003a0050
:101fb0000002eb001404980028029000040c780042
:101fc00019003700800278002520b2000000eb00e5
:101fd00024202000848f520016003a00a8009000b0
:101fe000808f50001300320018019000800f5100c4
:101ff00010003200480090008a000700180290008c
:10200000840f500003003200380290000403b30034
:10201000340498000002eb00140498002802900099
:10202000040c7800380090000002b2000100320079
:102030000080eb004f047800000006000200fa0068
:10204000889fbe00a0ff9f00010478003802900026
:10205000840278000504b200020032000000fb0098
:1020600035003700e202620005003a000403b300c5
:1020700034049800150498000080eb002e0037000f
:10208000d8049000e08f540006003a0012002000af
:10209000e68057004800900062000700190498008d
:1020a00023003700a8029000e08f520008003a0099
:1020b00055bf200025049800050c7800250020005d
:1020c00055049800150498000430a00034049800ca
:1020d00018019000a80090004800900051000700ef
:1020e000280290008082eb0015049800affa970058
:1020f000054a7800040ce8002ffa9700ea4f5200d6
:102100000b003a00380290000410b20008003200c0
:1021100018019000a80090004800900041000700be
:102120000002eb0014049800a8029000050c78004f
:102130002ffa97000400fb004f04be000080fa0055
:102140000000060000c0da00000006000a00fa00e5
:10215000e00f500027003a00d45f8000e10f5200ea
:10216000060032008723200066232000252320005c
:1021700004232000e08f530004003a00872220004f
:1021800066222000252220000422200000002800d2
:102190001400600003003a00800b7800070028005c
:1021a000148a7300020278000c0037008703e900ec
:1021b000950178006180610002003a00e08f5300d1
:1021c000faff3a0015007800e103600007003200d2
:1021d00096037800875878000402e900e00f520067
:1021e00002003200070a2000f1ff3700040051000e
:1021f0000800370024002000b4bf9f00c0bf9f002c
:10220000d1bf9f00e2bf9f006a805700cdff07004b
:102210006fb897000080fa000000060000c0da00e6
:10222000000006000a00fa00e20f500022003e0003
:10223000d45f8000e10f52000600320087232000a7
:10224000462320002423200005232000e08f530094
:1022500004003a0087222000462220002422200089
:1022600005222000000028001500600003003a004d
:10227000800b780007002800958a73000540200035
:102280009482620001003a0014a0a000820278004b
:1022900006003700940378000710b200fdff3200fb
:1022a000b103fb00070b78008502e900e08f5200c4
:1022b000f8ff3a000800370034002000b4bf9f0048
:1022c000c0bf9f00d1bf9f00e2bf9f006a80570040
:1022d000d2ff07006fb99700020078000080fa0073
:1022e000000006006022b800060220000000d000b6
:1022f0008180d2000482d2008582d2000000a0003a
:102300000202520083825a0003003100020242009e
:1023100083824a000000a1000603e900f3ff3a00af
:1023200000000600020ab900001bb9000200b80054
:10233000810042008100430000000600889fbe002b
:102340008a9fbe003004be002005be000404440085
:1023500085844c0006054d0087854d000898be0019
:102360000a90be000440e10005c8e10006d0e1008b
:1023700007d8e10002003100680040001008e800c2
:102380004f05be004f04be00000006001000fa001a
:10239000889fbe008a9fbe000605be000404be00e2
:1023a0003002be002003be00c4b79f00d5b79f0017
:1023b000e6b79f00f7b79f000802520089825a00d3
:1023c0000a035b008b835b0084bf9f0095bf9f0067
:1023d000a6bf9f00b7bf9f000498be000698be002e
:1023e000110020004fb29700dfb297006fb3970043
:1023f000ffb397000820e10009a8e1000ab0e1005e
:102400000bb8e100010039008000eb0010881000db
:102410004f05be004f04be000080fa000000060019
:102420001400fa00889fbe008a9fbe008c9fbe00e9
:102430003f0007000605be000404be000006eb00d6
:10244000ccb79f00bcb79f00acb79f009cb79f0064
:102450008cb79f000d0420004fb39700bfb29700c8
:10246000860343002fb29700e00f530004003d00a5
:102470003d0007000f004000b0ff070003003700d9
:10248000390007000f004000c0ff0700cfb29700df
:1024900095bf9f00e08f5200090035002b00070018
:1024a00014002000050020006033b8000000720016
:1024b0008180720002017300838173001c00070099
:1024c0000c06e8008d0f5600e3ff3a001fba970094
:1024d000e00f520005003d000802be000a03be00e6
:1024e00000fe2f000f00400094ff07004faa970046
:1024f000e00f520008003a000fb497009fb4970015
:102500002fb59700bfb59700d8b79f00e9b79f00d8
:10251000fab79f008bbf9f000c0007004f06be005c
:102520004f05be004f04be000080fa000000060008
:10253000010007000000060090b79f00a1b79f00b0
:10254000b2b79f00c3b79f0000000600010007005c
:10255000000006001fb09700afb097003fb1970092
:10256000cfb19700000006004f2bde0087037300f9
:10257000a7b79f004f23de008582420085027300cb
:1025800095b79f00ffaa97004f2bde000402420080
:102590000402730084b79f006faa97004f23de00e8
:1025a0008582420085027300f5af9f00e9ff0700b6
:1025b0004f18de000402420000027200e4af9f00e8
:1025c000e4ff07000000400081804800020149004c
:1025d00083814900d8ff07000802be000a03be003d
:1025e00000fe2f0000000600881f78001800200061
:1025f000881f78008aff07008f87e9004f04780062
:1026000000000600801feb0085ff07008f87e900b0
:1026100000000600889fbe008a9fbe00e00f5000a9
:10262000e08f5800e00f5900e08f59000c003d008a
:102630006044b8006055b8000000540081805c0020
:1026400002015d0083815d00180020001500070075
:1026500008003d00180007000004eb0005003700eb
:102660000004eb000f00070002003d00120007000d
:1026700018002000dcff0700e00f540006003200c5
:102680006022b8006033b8000000520081805a0018
:1026900002015b0083815b004f05be004f04be005a
:1026a00000000600e00f5200e08f5a00e00f5b00d0
:1026b000e08f5b00000006006044b8006055b80081
:1026c0000402540085825c0006035d0087835d0080
:1026d00000000600889fbe008a9fbe008c1f780005
:1026e000e00f5000e08f5800e00f5900e08f5900d4
:1026f0000d003d006044b8006055b8000000540073
:1027000081805c0002015d0083815d001c0020006f
:102710000820e10009a8e1000ab0e1000bb8e100df
:102720000d003d00080037000006eb00e00f5200ee
:10273000e08f5a00e00f5b00e08f5b0006003d0079
:102740006044b8006055b8000402540085825c0003
:1027500006035d0087835d00aaff0700e00f5600b7
:10276000060032006022b8006033b800000052005a
:1027700081805a0002015b0083815b004f06780074
:102780004f05be004f04be0000000600889fbe003b
:102790008a9fbe008c1f78000006eb00e00f5000ff
:1027a000e08f5800e00f5900e08f590007003d000e
:1027b0006044b8006055b8000000540081805c009f
:1027c00002015d0083815d001c002000e00f5200cb
:1027d000e08f5a00e00f5b00e08f5b0007003d00d8
:1027e0006044b8006055b8000402540085825c0063
:1027f00006035d0087835d000c00a2000c0007004b
:10280000e00f5600060032006022b8006033b800c6
:102810000000520081805a0002015b0083815b004e
:102820004f0678004f05be004f04be0000000600b2
:10283000889fbe008a9fbe008c9fbe000404b80023
:102840000506b8008904460060854e000606b800fb
:102850000a054600e0854e000706b8008b054600d5
:10286000040eb800890446000a854e00e0854d003c
:10287000050eb8000a0546008b854e00060eb8000e
:102880008b0546000416b8000a0546008b854e00ed
:102890000516b8008b054600041eb8008b054600df
:1028a0000800be000a01be004f06be004f05be0074
:0828b0004f04be000000060009
:020000040000fa
:1028b8004d4500004f5700000d0a0000004200007f
:1028c80049540000202500006420000049530000fe
:1028d80020480000490d00000a000000424900009d
:1028e8005420000025640000204900005320000007
:1028f8004c4f00000d0a0000004400004154000045
:10290800453a0000200000000d0a000000540000b5
:10291800494d0000453a00002000000054490000dd
:102928004d4500002053000045540000204600009b
:102938004f5200004d410000543a0000206800004a
:10294800683a00006d6d00003a730000733a0000a9
:10295800776400003a440000443a00004d4d0000fe
:102968003a590000590d00000a0000007764000081
:1029780028770000656500006b2000006461000096
:10298800792900003a200000302000003d20000096
:10299800537500006e640000617900002c2000006f
:1029a800312000003d2000004d6f00006e640000e3
:1029b800617900002c20000065740000632e00007f
:1029c8000d0a000000250000643a0000256400009c
:1029d8003a250000643a0000256400003a2500000a
:1029e800643a0000256400003a25000064000000f5
:1029f80045520000523a00002046000041490000bc
:102a08004c45000044200000544f000020530000b3
:102a18004554000020520000544300000d0a0000f5
:102a28000072000074630000536500007420000009
:102a38007265000074750000726e0000732000005b
:102a4800535500004343000045530000530d000058
:102a58000a000000526500006c6100007920000047
:102a68002564000020490000532000004f4e00005c
:102a78000d0a000000520000656c0000617900003a
:102a8800202500006420000069730000204f00002a
:102a9800464600000d0a0000004e00006f200000ae
:102aa800737500006368000020720000656c000008
:102ab800617900000d0a00000054000075720000e2
:102ac8006e6900006e670000206f00006e20000035
:102ad800726500006c610000792000002564000028
:102ae8000d0a000000540000757200006e690000b5
:102af8006e670000206f000066660000207200000c
:102b0800656c00006179000020250000640d00005c
:102b18000a0000000d0a00004e6f00002069000046
:102b28006e7000007574000020630000686100008a
:102b380072730000206f00006e20000073650000b3
:102b480072690000616c0000202300003100000061
:102b58000d0a00004e6f0000206900006e70000032
:102b68007574000020630000686100007273000043
:102b7800206f00006e20000073650000726900007d
:102b8800616c000020230000320000005375000033
:102b98006e640000617900002c200000004d0000e8
:102ba8006f6e000064610000792c000020000000b6
:102bb800547500006573000064610000792c000002
:102bc8002000000057650000646e00006573000077
:102bd80064610000792c00002000000054680000a7
:102be8007572000073640000617900002c200000f9
:102bf800004600007269000064610000792c000042
:102c08002000000053610000747500007264000029
:102c1800617900002c200000005b00003f3f0000ad
:102c28003f5d000064610000792c00002000000076
:102c38004a6100006e750000617200007920000092
:102c480000460000656200007275000061720000b5
:102c580079200000004d00006172000063680000e8
:102c68002000000041700000726900006c20000024
:102c7800004d000061790000200000004a75000046
:102c88006e650000200000004a7500006c790000a5
:102c98002000000041750000677500007374000093
:102ca800200000005365000070740000656d00008e
:102cb8006265000072200000004f0000637400008d
:102cc8006f62000065720000200000004e6f000077
:102cd800766500006d62000065720000200000004b
:102ce80044650000636500006d62000065720000c5
:102cf800200000005b3f00003f3f00005d6d0000ca
:102d08006f6e00007468000020000000253000008d
:102d1800326400002c200000003200003025000042
:102d280030320000640000002530000032640000ea
:102d38003a25000030320000643a000025300000d7
:102d48003264000000000000313500003a31000014
:102d5800353a000031370000004600006562000087
:102d680020310000302000003230000031340000f3
:102d7800000d00000a730000774600004f43000072
:102d8800452000004d65000064690000756d000075
:102d9800205600006f6c0000746100006765000039
:102da800204300006f6e000076650000727400001a
:102db80065720000204200006f610000726400002c
:102dc80020420000756900006c740000206f00004c
:102dd8006e200000257300002061000074200000b0
:102de800257300000d0a0000000d00000a4d0000c8
:102df800564300006f6e000076200000426f00000e
:102e080061720000642000007365000072690000b0
:102e1800616c0000207000006f72000074200000d8
:102e2800233100000d0a0000000d00000a4d0000cb
:102e3800564300006f6e000076200000426f0000cd
:102e48006172000064200000736500007269000070
:102e5800616c0000207000006f7200007420000098
:102e6800233200000d0a00000020000009000000c5
:102e78004552000052200000253000003464000054
:102e88000d0a000000520000445900000d0a00001d
:102e980000000000474500005400000053450000b2
:102ea80054000000434c000045410000527c0000e3
:102eb800434c000052000000484500004c4c000004
:102ec8004f2000004b4900005454000059000000f6
:102ed800000000004e9700005a2900005297000099
:102ee8006e290000569700008229000060970000b4
:102ef800962900006c97000000000000444900007b
:102f08004e000000444f00005554000000540000db
:102f1800494d000045000000524500004c410000aa
:102f280059000000534500005231000000530000d2
:102f3800455200003200000082970000a8290000d6
:102f480086970000e62900008b970000242a0000dd
:102f580090970000642b000096970000122d000047
:102f68009b9700004e2d00006c97000000000000a9
:102f7800524500004c410000594f00004e0000002f
:102f8800524500004c410000594f000046460000e1
:102f98000000000086970000642a00008b9700005c
:102fa8007e2a0000bc970000ca2b0000c4970000ce
:102fb800662c0000969700001a2b00009b970000d3
:102fc800322b00006c97000000000000869700007c
:102fd8004a2b00006c970000000000002009000048
:102fe80000200000003000003132000033340000bf
:0c2ff800353600003738000039000000ba
:020000040000fa
:103004000000fa002c03a8002c23a8002c43a800dd
:103014002c63a8002c83a8002ca3a8002cc3a80010
:103024002ce3a8002d03a8002d23a8002d43a800fd
:103034002d63a8002d83a8002da3a8002dc3a800ec
:103044002de3a800c842a900c862a900c882a9004b
:10305400c8a2a900c8c2a900c8e2a900c902a9005f
:10306400c922a900c942a900c962a900c982a9004c
:10307400c9a2a900c9c2a900c9e2a900d8c2a9006d
:10308400d8e2a900d902a900d922a900d942a900ed
:10309400d962a900e802a900e822a900e842a9002f
:1030a400e862a900e882a900e8a2a900e8c2a90090
:1030b400f0c2a900e002a800e022a800e042a800b3
:1030c400e062a800e082a800e0a2a800e0c2a80094
:1030d400f042a800f062a80000000000cc42a90061
:1030e40000000000cc62a90000000000cc82a9000e
:1030f40000000000cca2a90000000000ccc2a9007e
:1031040000000000cce2a90000000000cd02a900ec
:1031140000000000cd22a90000000000cd42a9005b
:1031240000000000cd62a90000000000cd82a900cb
:1031340000000000cda2a90000000000cdc2a9003b
:1031440000000000cde2a90000000000dcc2a800dd
:1031540000000000dce2a80000000000dd02a8007e
:1031640000000000dd22a80000000000dd42a800ed
:1031740000000000dd62a80000000000ec02a900cd
:1031840000000000ec22a90000000000ec42a800ae
:1031940000000000ec62a80000000000ec82a9001e
:1031a40000000000eca2a90000000000ecc2a9008d
:1031b40000000000f4c2a900000000000080fa0032
:1031c400000006000400fa00000f780011079800c0
:1031d4001e029000e00f5200020032001400200092
:1031e40014079800000000001e027800cfa2de0041
:1031f400b601200007002000860f5200878f5a0076
:103204006b013e00046001001b00370026003700fc
:10321400310037003c0037004700370052003700c8
:103224005d00370068003700730037007e00370008
:1032340089003700940037009f003700aa00370048
:10324400b4003700bf003700ca003700d50037008c
:10325400e0003700eb003700f600370000013700cc
:103264000b01370016013700210137002c0137000c
:1032740037013700420137001e02900004427800f3
:10328400614262000482fb00610262004222dd00ae
:1032940066168000b5ff2f00850263000482720069
:1032a40064168800430137001e029000044278002f
:1032b400614262000482fb00610262004322dd007d
:1032c4006616800075ff2f00850263000482720079
:1032d40064168800370137001e029000044278000b
:1032e400614262000482fb00610262004422dd004c
:1032f40066168000f5fe2f008502630004827200ca
:10330400641688002b0137001e02900004427800e6
:10331400614262000482fb00610262004522dd001a
:1033240066168000f5fd2f0085026300048272009a
:10333400641688001f0137001e02900004427800c2
:10334400614262000482fb00610262004622dd00e9
:1033540066168000f5fb2f0085026300048272006c
:1033640064168800130137001e029000044278009e
:10337400614262000482fb00610262004722dd00b8
:1033840066168000f5f72f00850263000482720040
:1033940064168800070137001e029000044278007a
:1033a400614262000482fb00610262004822dd0087
:1033b40066168000f5ef2f00850263000482720018
:1033c40064168800fb0037001e0290000442780057
:1033d400614262000482fb00610262004922dd0056
:1033e40066168000f5df2f008502630004827200f8
:1033f40064168800ef0037001e0290000442780033
:10340400614262000482fb00610262004a22dd0024
:1034140066168000f5bf2f008502630004827200e7
:1034240064168800e30037001e029000044278000e
:10343400614262000482fb00610262004b22dd00f3
:1034440066168000f57f2f008502630004827200f7
:1034540064168800d70037001e02900004427800ea
:10346400614262000482fb00610262004c22dd00c2
:1034740066168000f5ff2e00850263000482720048
:1034840064168800cb0037001e02900004427800c6
:10349400614262000482fb00610262004d22dd0091
:1034a40066168000f5ff2d00850263000482720019
:1034b40064168800bf0037001e02900004427800a2
:1034c400614262000482fb00610262004e22dd0060
:1034d40066168000f5ff2b008502630004827200eb
:1034e40064168800b30037001e029000044278007e
:1034f400614262000482fb004f22dd0066168000f8
:10350400f5ff2700850263000482720064168800b8
:10351400a80037001e029000044278006142620055
:103524000482fb00610262004622dd00e616800090
:10353400f5fb2f008502630004827200e416880004
:103544009c0037001e029000044278006142620031
:103554000482fb00610262004722dd00e61680005f
:10356400f5f72f008502630004827200e4168800d8
:10357400900037001e02900004427800614262000d
:103584000482fb00610262004822dd00e61680002e
:10359400f5ef2f008502630004827200e4168800b0
:1035a400840037001e0290000442780061426200e9
:1035b4000482fb00610262004922dd00e6168000fd
:1035c400f5df2f008502630004827200e416880090
:1035d400780037001e0290000442780061426200c5
:1035e4000482fb00610262004a22dd00e6168000cc
:1035f400f5bf2f008502630004827200e416880080
:103604006c0037001e0290000442780061426200a0
:103614000482fb00610262004b22dd00e61680009a
:10362400f57f2f008502630004827200e41688008f
:10363400600037001e02900004427800614262007c
:103644000482fb006102620066178000e5ff2f0020
:1036540085026300048272006417880055003700f5
:103664001e02900004427800614262000482fb0062
:10367400610262000402420066178000d5ff2f0039
:1036840085026300048272006417880049003700d1
:103694001e02900004427800614262000482fb0032
:1036a400610262004222dd0066178000b5ff2f0030
:1036b4008502630004827200641788003d003700ad
:1036c4001e02900004427800614262000482fb0002
:1036d400610262004322dd006617800075ff2f003f
:1036e4008502630004827200641788003100370089
:1036f4001e02900004427800614262000482fb00d2
:10370400610262004422dd0066178000f5fe2f008e
:103714008502630004827200641788002500370064
:103724001e02900004427800614262000482fb00a1
:10373400610262004522dd0066178000f5fd2f005e
:103744008502630004827200641788001900370040
:103754001e02900004427800614262000482fb0071
:10376400610262004622dd0066178000f5fb2f002f
:103774008502630004827200641788000d0037001c
:103784001e02900004427800614262000482fb0041
:10379400610262004622dd00a6178000f5fb2f00bf
:1037a4008502630004827200a417880001003700b8
:1037b400000000000080fa00000006000200fa0089
:1037c400000f7800000000000002eb00f4578800ae
:1037d4001e027800cfa2de00b60120000700200000
:1037e400860f5200878f5a00a9003e000460010032
:1037f4001b0037001f003700230037002700370065
:103804002b0037002f003700330037003700370014
:103814003b0037003f0037004300370047003700c4
:103824004b0037004f003700530037005700370074
:103834005b0037005f003700630037006700370024
:103844006b0037006f0037007300370077003700d4
:103854007b0037007f003700830037008700370084
:10386400641680004222de00614262000482fb0092
:1038740088003700641680004322de006142620043
:103884000482fb0083003700641680004422de00bb
:10389400614262000482fb007e00370064168000ef
:1038a4004522de00614262000482fb007900370099
:1038b400641680004622de00614262000482fb003e
:1038c40074003700641680004722de006142620003
:1038d4000482fb006f003700641680004822de007b
:1038e400614262000482fb006a00370064168000b3
:1038f4004922de00614262000482fb006500370059
:10390400641680004a22de00614262000482fb00e9
:1039140060003700641680004b22de0061426200c2
:103924000482fb005b003700641680004c22de003a
:10393400614262000482fb00560037006416800076
:103944004d22de00614262000482fb005100370018
:10395400641680004e22de00614262000482fb0095
:103964004c003700641680004f22de0004427800c9
:103974000482fb0047003700e41680004622de0084
:10398400614262000482fb0042003700e4168000ba
:103994004722de00614262000482fb003d003700e2
:1039a400e41680004822de00614262000482fb00cb
:1039b40038003700e41680004922de0061426200cc
:1039c4000482fb0033003700e41680004a22de0044
:1039d400614262000482fb002e003700e41680007e
:1039e4004b22de00614262000482fb0029003700a2
:1039f4006417800004427800614262000482fb0084
:103a040024003700641780000402d1006142620080
:103a14000482fb001f003700641780004222de008e
:103a2400614262000482fb001a00370064178000c0
:103a34004322de00614262000482fb00150037006d
:103a4400641780004422de00614262000482fb00ad
:103a540010003700641780004522de0061426200d6
:103a64000482fb000b003700641780004622de004e
:103a7400614262000482fb0006003700a417800044
:103a84004622de00614262000482fb00010037002e
:103a94000002eb00040078000080fa000000060039
:103aa4000600fa002007980014002000140798006c
:103ab4000002eb00040f78000a003700ae02900009
:103ac4001e02900004826200840078001e007800c8
:103ad400bcfd07001e029000040242001407980077
:103ae4001e0fe8001e027800ff0f5200f3ff34009f
:103af4000080fa00000006000600fa00140020000e
:103b0400140798000002eb00240798000002eb0061
:103b1400040f78000d0037001e00780027ff07000f
:103b240000027800e00f520004003200ae02900060
:103b34001e02900004824200240798001e02900096
:103b440004024200140798001e0fe8001e027800c9
:103b5400ff0f5200f0ff34002e02900004007800a2
:103b64000080fa00000006000200fa00000f78004e
:103b7400000000000002eb00f45788001e027800e9
:103b8400cfa2de009600200007002000860f52001e
:103b9400878f5a003d003e00046001000900370091
:103ba4000d003700110037001500370019003700e9
:103bb4001d00370021003700250037002900370099
:103bc4002d0037001417800004427800614262001f
:103bd4000482fb002e003700141780000402d10079
:103be400614262000482fb00290037001417800040
:103bf4004222de00614262000482fb00240037009e
:103c0400141780004322de00614262000482fb003c
:103c14001f003700141780004422de006142620056
:103c24000482fb001a003700141780004522de00ce
:103c3400614262000482fb00150037001417800003
:103c44004622de00614262000482fb00100037005d
:103c5400141780004722de00614262000482fb00e8
:103c64000b003700941780004222de00614262009c
:103c74000482fb0006003700941780004322de0014
:103c8400614262000482fb00010037000002eb0085
:103c9400040078000080fa00000006000600fa0024
:103ca40014002000140798000002eb002407980079
:103cb4000002eb00040f78000d0037001e007800ae
:103cc400a9ff070000027800e00f52000400320050
:103cd400ae0290001e029000048242002407980065
:103ce4001e02900004024200140798001e0fe80010
:103cf4001e027800ef0f5200f0ff34002e029000f5
:103d0400040078000080fa00000006000200fa00b7
:103d14002474200014427800044378000614a000a0
:103d2400064f78001e4278008483fb006404200060
:103d340076052000207420000448780006487800a6
:103d4400074878004207a80055052000353b880045
:103d5400a50a2000353b880027a6a80027e6a8006e
:103d640027a6a9000080fa00000006000c00fa0053
:103d7400881f7800500798005e029000544290001b
:103d84000482fb0084007800100020004402070035
:103d940000027800140798005e02900064429000cc
:103da4000482fb00840078000000eb003c02070062
:103db400000278009e0290000482420014079800da
:103dc4005e029000344290000482fb00840078007c
:103dd4001000200032020700000278002407980037
:103de4005e029000444290000482fb00840078004c
:103df4000000eb002a02070000027800ae029000e7
:103e040004824200240798005e029000144290004d
:103e14000482fb00840078001000200020020700c8
:103e240000027800340798005e029000244290005b
:103e34000482fb00840078000000eb0018020700f5
:103e440000027800be029000048242003407980009
:103e54005e029000144278000482fb008400780023
:103e64000000eb000e0207000002780044079800ef
:103e740058052000383b8800a80a2000383b8800f9
:103e840027a6a800343180000480a1000490a1007a
:103e9400343188001e0290002431880034318000bf
:103ea4000480a0000490a100343188002e02900008
:103eb40024318800343180000480a1000490a000e3
:103ec400343188003e02900024318800343180006f
:103ed4000480a0000490a000343188004e029000b9
:103ee4002431880014002000040f7800343180004d
:103ef4000480a1000490a1003431880024318000a2
:103f04009e029000848f5200020032000002eb00f7
:103f1400040f7800343180000480a0000490a100d4
:103f24003431880024318000ae029000848f520026
:103f3400020032000002eb00040f780034318000ec
:103f44000480a1000490a000343188002431800052
:103f5400be029000848f5200020032000002eb0087
:103f6400040f7800343180000480a0000490a00085
:103f74003431880024318000ce029000848f5200b6
:103f8400020032000002eb00040f780027a6a9000b
:103f94001e027800040078004f0478000080fa00c4
:103fa400000006000e00fa00600798005405200087
:103fb400343b8800a40a2000343b880027a6a800cc
:103fc4000002eb00040f7800520037003431800007
:103fd4000480a1000490a1003431880024318000c1
:103fe40024079800343180000480a0000490a100cc
:103ff4003431880024318000340798003431800043
:104004000480a1000490a000343188002431800091
:1040140044079800343180000480a0000490a0007c
:1040240034318800243180005407980035318000f1
:104034000480200004826200e00f52000400320079
:10404400ee02900014c0b300f4429800030037005d
:10405400ee0290000042eb00f442980014002000ad
:1040640014079800343180000480a1000490a1005a
:104074003431880024318000ae029000848f5200d5
:10408400020032000002eb00140798003431800073
:104094000480a0000490a100343188002431800001
:1040a400be029000848f5200020032000002eb0036
:1040b40014079800343180000480a1000490a0000b
:1040c4003431880024318000ce029000848f520065
:1040d400020032000002eb00140798003431800023
:1040e4000480a0000490a0003431880024318000b2
:1040f400de029000848f5200020032000002eb00c6
:10410400140798001e029000e00f520005003a00c8
:104114001e0fe8001e027800e20f5200abff3400cd
:10412400010037000000000027a6a9001e0290002d
:10413400e00f520032003200de0090000000eb007d
:104144007f0107000002780004427800ee0290002c
:10415400844a7800ce009000100020007801070007
:104164000002780004427800ee0290009442980025
:10417400ce0090000000eb007101070000027800ff
:1041840004427800ee029000a4429800be00900021
:10419400100020006a010700000278000442780041
:1041a400ee029000b4429800be0090000000eb00c4
:1041b400630107000002780004427800ee029000d8
:1041c400c4429800ae009000100020005c0107007b
:1041d4000002780004427800ee029000d442980075
:1041e400ae0090000000eb005501070000027800cb
:1041f40004427800ee029000e44298001800370070
:10420400ee0290000042eb00844a7800ee02900037
:104214000042eb0094429800ee0290000042eb0052
:10422400a4429800ee0290000042eb00b4429800d1
:10423400ee0290000042eb00c4429800ee029000af
:104244000042eb00d4429800ee0290000042eb00e2
:10425400e4429800ee0290000042eb00f442980021
:104264001e029000040078000080fa00000006009e
:104274000c00fa0040079800510798004e02900085
:10428400344290000482fb00cfa2de0066002000ce
:1042940007002000860f5200878f5a002b003e0033
:1042a40004600100060037000a0037000e003700e2
:1042b40012003700160037001a0037001e003700be
:1042c40092002000a15c29005e0090000cf1070020
:1042d4002300370092002000315d29005e00900029
:1042e40007f107001e003700a2002000c15d29006d
:1042f4005e00900002f1070019003700c2002000a0
:10430400615e29005e009000fdf007001400370094
:10431400b2002000215f29005e009000f8f0070041
:104324000f00370092002000d15f29005e0090004a
:10433400f3f007000a003700b20020006160290092
:104344005e009000eef0070005003700b200200088
:10435400116129005e009000e9f0070000000000f0
:104364004e029000144290000482fb006123b900c5
:104374000082eb008082eb000602420087824a0042
:10438400b600200007002000860f5200878f5a00d5
:1043940085003e00046001000b0037001400370064
:1043a4001d003700260037002f0037003800370083
:1043b400410037004a003700530037005c003700e3
:1043c400650037006e0037005e009000def00700e5
:1043d40000027800de029000048242009200200075
:1043e400c161290004007800c5f007007800370097
:1043f4005e009000d4f0070000027800de02900016
:1044040004824200a20020005162290004007800c6
:10441400bbf007006e0037005e009000caf0070092
:1044240000027800de029000048242007200200044
:10443400f162290004007800b1f00700640037003d
:104444005e009000c0f0070000027800de029000d9
:104454000482420072002000616329000400780095
:10446400a7f007005a0037005e009000b6f007007e
:1044740000027800de029000048242005200200014
:10448400d1632900040078009df007005000370034
:104494005e009000acf0070000027800de0290009d
:1044a4000482420062002000216429000400780094
:1044b40093f00700460037005e009000a2f007006a
:1044c40000027800de0290000482420062002000b4
:1044d400816429000400780089f007003c0037005b
:1044e4005e00900098f0070000027800de02900061
:1044f4000482420082002000e16429000400780064
:104504007ff00700320037005e0090008ef0070055
:1045140000027800de02900004824200b200200013
:10452400616529000400780075f007002800370051
:104534005e00900084f0070000027800de02900024
:1045440004824200920020001166290004007800d1
:104554006bf007001e0037005e0090007af0070041
:1045640000027800de02900004824200a2002000d3
:10457400a16629000400780061f0070014003700e8
:104584005e00900070f0070000027800de029000e8
:1045940004824200a2002000416729000400780040
:1045a40057f007000a0037005e00900066f007002d
:1045b40000027800de02900004824200c200200063
:1045c400e1672900040078004df0070000000000b6
:1045d4004e029000244290000482fb00841f780065
:1045e400a4682900841f78000e007800f1f1070008
:1045f400e48757008e0078005e00900047f00700c3
:104604004e029000144278000482fb00841f78005c
:1046140014692900841f78000e007800e5f1070072
:10462400e48757008e0078005e0090003bf007009e
:1046340014002000040078000080fa000000060046
:104644000400fa00000f7800110798001e02780099
:10465400644290000483fb001e02780054429000e0
:104664008482fb001e027800444290000482fb0016
:10467400861f7800851f7800841f780084692900cc
:10468400841f78001e009000caf10700e8875700d5
:1046940014002000040078000080fa0000000600e6
:1046a4000800fa002007980031079800be02900025
:1046b400a4002000809fbe00110009008482d8005d
:1046c40000027800810278004f00be002447980061
:1046d4002e429000650f200005a2b9000402780064
:1046e400844278003e0290000442780004c24200f2
:1046f400344798002e4290000482fb00040f780097
:104704001e0278004422dd00040f78003e4290002f
:104714000482fb001e0f42002e029000e00f5200a4
:10472400030032001e0278004822dd00040f7800e6
:104734001e027800040078000080fa0000000600e1
:104744000a00fa0030079800410798003e029000e2
:10475400e00f520007003200ce02900004f02f0058
:10476400048f62001e0278004822de00040f7800e5
:1047740003003700ce029000f40f2000048f620083
:104784001e0278008442780004cfb30004c26200a1
:10479400244798002e4290000482fb004422de004d
:1047a400244798001e027800044278006f42620099
:1047b400344798002e4290000482fb00240798009e
:1047c4002e0290006a22b90004027800240798009f
:1047d4003e4290000482fb00ae029000048242003c
:1047e400240798002e029000040078000080fa004c
:1047f400000006000200fa000002eb00040f78003b
:104804003d003700858120001e0278004722dd002c
:10481400848242001e0278004323dd0004802000cd
:1048240004024300050a78001e027800c322dd005a
:1048340024802000048242008002eb00050a7800f4
:104844001e027800c322dd0044802000048242005e
:104854008002eb00050a78001e027800c322dd0006
:104864006480200004824200f5072000050a7800d5
:10487400659b20001e0278004522dd0084824200f0
:104884001e0278004323dd00e49920000402430063
:10489400050a78001e027800c322dd00049a200075
:1048a400048242008002eb00050a78001e027800b0
:1048b400c322dd00249a2000048242008002eb001f
:1048c400050a78001e027800c322dd00449a200005
:1048d40004824200f5012000050a78001e027800d7
:1048e4008402420084992000048242008002eb008a
:1048f400050a78001e0fe8001e027800e20f52003d
:10490400c0ff3400b40020004411880021e2a80054
:1049140020a2a9002062a900041180000410a100b3
:104924000420a100041188002002a90004402000f2
:10493400141188008560a9008580a90044058000c1
:1049440004c0a10004d0a00004e0a0004405880035
:10495400540580000400a1000410a0000420a1005c
:10496400540588009560a8009580a900b400200033
:10497400c411880031e2a80030a2a9003062a90065
:10498400841180000410a1000420a1008411880077
:104994003002a900044020009411880087c0a900b7
:1049a40087e0a900940580000480a1000490a00081
:1049b40004a0a000940588009405800004c0a10010
:1049c40004d0a00004e0a1009405880097c0a800ca
:1049d40097e0a900b4002000c412880051e2a800a6
:1049e40050a2a9005062a900841280000410a10002
:1049f4000420a100841288005002a9000440200071
:104a0400941288008e40a9008e60a900640680007c
:104a14000480a1000490a00004a0a0006406880003
:104a24006406800004c0a10004d0a00004e0a1003a
:104a3400640688009e40a8009e60a9000080fa00d9
:104a4400000006000600fa001007980021079800ed
:104a54001e029000e30f520003003c001e0290006f
:104a6400e00f520005003c00ae0290000042eb0053
:104a7400844a78000002eb000d0037002b08070081
:104a84001e0290000402e900c322dd00048020001d
:104a940004824200840078002e0090007a07070008
:104aa40000027800040f78002a0807001e0278002c
:104ab400040078000080fa00000006000600fa00f6
:104ac400100798004147980014002000040f780054
:104ad4001e029000e20f52001c003200e30f52004d
:104ae40032003200e10f520047003a00a504800072
:104af4000400210004826200e00f520005003a0025
:104b0400151180000420200004826200e00f52008e
:104b14000900320005080700e19920004e4090008a
:104b24003d07070000027800040f78009580a80074
:104b340008080700030037004e4290000482fb007f
:104b4400241188001e02780030003700b50480006c
:104b54000400280004826200e00f520005003a00bd
:104b6400951180000420200004826200e00f5200ae
:104b740009003200ed070700619a20004e409000c2
:104b84002507070000027800040f780097e0a800ca
:104b9400f0070700030037004e4290000482fb0038
:104ba400a41188001e02780018003700f404800065
:104bb40068026200e00f520005003a00951280007e
:104bc4000420200004826200e00f52000900320039
:104bd400d6070700e19a20004e4090000e07070018
:104be40000027800040f78009e60a800d90707002f
:104bf400030037004e4290000482fb00a412880098
:104c04001e027800010037000002eb000400780067
:104c14000080fa00000006000600fa001007980061
:104c2400210798000002eb00040f78000b00370006
:104c34001e027800ae029000048242001442780002
:104c4400844078001e0090009cff0700000278005a
:104c5400e00f5200010032001e0fe8001e0278002f
:104c6400ae0290000482420014427800e04f5200e9
:104c7400efff3a000002eb00040078000080fa0025
:104c8400000006000400fa00100798001e029000bd
:104c9400e20f520006003200e30f52000600320019
:104ca400e10f5200060032000002eb001100370051
:104cb400000000000300370000000000010037007e
:104cc40000000000990707001e0290000402e9009a
:104cd400c322dd0004802000048242000400780026
:104ce4001407070000027800040f780099070700f2
:104cf4001e027800040078000080fa00000006001c
:104d04000400fa00100798001e029000e20f5200ff
:104d14000a003200e30f52000e003200e10f52008d
:104d240012003a00141180004922de006142620040
:104d34000482fb00040f78000e00370094118000f9
:104d44004922de00614262000482fb00040f780005
:104d540008003700941280004922de00614262009c
:104d64000482fb00040f78000200370014002000c6
:104d7400040f78001e027800040078000080fa0016
:104d8400000006000200fa00000f78001e027800fe
:104d9400e20f52000a003200e30f52000e0032000c
:104da400e10f520012003a001e0278008402420011
:104db4008499200004824200140278000d00370018
:104dc4001e0278008402420084992000048242007a
:104dd40014027800070037001e02780084024200a3
:104de40084992000048242001402780001003700f4
:104df4000002eb00040078000080fa0000000600c6
:104e04000200fa00000f78001e027800e20f520040
:104e140005003200e30f520005003200e10f52009a
:104e24000b003a00030037000000000001003700c7
:104e3400000000001e0278008402420084992000d1
:104e4400048242008002eb00050a7800010037006a
:104e5400000000000080fa00000006000400fa00d0
:104e6400100798001e029000e20f52000500320065
:104e7400e30f520005003200e10f520032003a0005
:104e840003003700000000000100370000000000ac
:104e9400260707001e0290000402e900c322dd0079
:104ea4000480200004824200040078009706070072
:104eb4001e029000e20f520011003200e30f520074
:104ec40018003200e10f5200040032001b003700ca
:104ed40034118000040f7800010037000000000046
:104ee4001411800061026200e00f5200f8ff3a00e2
:104ef40012003700b4118000040f7800010037005d
:104f0400000000009411800061026200e00f520072
:104f1400f8ff3a0009003700b4128000040f78004b
:104f2400010037000000000094128000610262005a
:104f3400e00f5200f8ff3a000000000005070700e8
:104f44000000000001003700000000000080fa00ab
:104f5400000006000200fa00000f78001e0278002c
:104f6400e20f520008003200e30f52000a00320040
:104f7400e10f52000e003a002342a9000000000095
:104f84002342a800000000003342a90000000000f2
:104f94003342a800000000005342a90000000000b2
:104fa4005342a80000000000000000000100370088
:104fb400000000000080fa00000006003600f8003f
:104fc400809fbe00829fbe00849fbe00869fbe005d
:104fd4000200fa00151180000420200004826200ff
:104fe400e00f52000b003a00e19920000e00780017
:104ff4002506070000027800e00f5200040032008a
:105004001e4278000482fb0024118800010037004e
:105014009580a900000000008580a9000080fa00a6
:105024004f03be004f02be004f01be004f00be0042
:105034003600f90000400600849fbe000000fa001c
:1050440015003700144080008402e80034408000da
:105054008482620024408000848f520003003a005e
:1050640014002000c44c88000b0037000540800069
:10507400144080008482420034118000044278008d
:10508400844a7800144080008402e80034408000a0
:1050940004826200144088001411800061026200de
:1050a400e00f5200e7ff3a008560a9000080fa0093
:1050b4004f02be00004006003600f800809fbe008c
:1050c400829fbe00849fbe00869fbe000200fa003d
:1050d400951180000420200004826200e00f520039
:1050e4000b003a00619a20000e007800e6050700e4
:1050f40000027800e00f5200040032001e427800e3
:105104000482fb00a41188000100370097e0a90085
:105114000000000087e0a9000080fa004f03be00f1
:105124004f02be004f01be004f00be003600f90022
:1051340000400600849fbe000000fa0015003700fe
:10514400544080008402e80074408000848262003d
:1051540064408000848f520003003a001400200051
:10516400d44c88000b003700454080005440800038
:1051740084824200b411800004427800844a78009a
:10518400544080008402e80074408000048262007d
:10519400544088009411800061026200e00f5200c4
:1051a400e7ff3a0087c0a9000080fa004f02be0062
:1051b400004006003600f800809fbe00829fbe00bb
:1051c400849fbe00869fbe000200fa0095128000f4
:1051d4000420200004826200e00f52000b003a0019
:1051e400e19a20000e007800a7050700000278006d
:1051f400e00f5200040032001e4278000482fb00db
:10520400a4128800010037009e60a900000000007d
:105214008e60a9000080fa004f03be004f02be005a
:105224004f01be004f00be003600f90000400600ea
:10523400849fbe000000fa001500370094408000ef
:105244008402e800b440800084826200a4408000ac
:10525400848f520003003a0014002000e44c8800bc
:105264000b00370085408000944080008482420017
:10527400b412800004427800844a7800944080008c
:105284008402e800b44080000482620094408800f4
:105294009412800061026200e00f5200e7ff3a00be
:1052a4008e40a9000080fa004f02be0000400600b4
:1052b4000200fa00000f780052002000017a290051
:1052c4001e007800a604070000027800040078009d
:1052d4000080fa00000006000200fa00000f7800c7
:1052e40052002000e17c29001e0078009c04070085
:1052f40000027800040078000080fa000000060034
:105304000200fa00000f780052002000a17e29005c
:105314001e00780092040700000278000400780060
:105324000080fa00000006000200fa00000f780076
:10533400c14529003000200037fe07000002eb00c1
:10534400040078000080fa00000006000400fa005f
:10535400100798001e009000caec070000027800b5
:10536400040f78001e007800fff90700000278009f
:10537400e00f5200070032009e1f780034462900d7
:10538400841f780060a120008aee0700e48757009c
:10539400060037009e1f780024472900841f7800e8
:1053a40060a1200083ee0700e487570061a120007c
:1053b4003000200018fe07000002eb000400780013
:1053c4000080fa00000006000400fa0010079800ac
:1053d4001e009000abec070000027800040f780078
:1053e4001e007800f5f8070000027800e00f520074
:1053f400070032009e1f780034462900841f78007d
:1054040060a120006bee0700e48757000600370018
:105414009e1f780024472900841f780060a1200083
:1054240064ee0700e487570061a1200030002000eb
:10543400f9fd07000002eb00040078000080fa0088
:10544400000006000a00fa00400798000e007800e9
:10545400d4fa070061a120000e00780084fb070045
:105464001148290030002000ebfd070061a1200055
:1054740030002000e8fd07008148290030002000aa
:10548400e5fd070061a120000e0078006cfc070018
:10549400b148290030002000dffd070061a1200091
:1054a40030002000dcfd0700814829003000200086
:1054b400d9fd07000002eb00040078000080fa0028
:1054c400000006000400fa00100798001e00900077
:1054d4006cec070000027800040f78001100200033
:1054e4001e00780037f707000002eb000400780084
:1054f4000080fa00000006001800fa00300f98003f
:105504003e0a900014427800e04f520008003a002e
:105514002149290030002000bffd0700a14b2900cc
:1055240030002000bcfd07000002eb003d00370006
:1055340068024700841f7800680247000482e8007c
:10554400841f78006802470064024200841f7800c8
:105554006802470066024200841f78006802470020
:105564006c024200841f7800680247006a0242000d
:10557400841f78006802470068024200841f780094
:10558400744e2900841f78003e08900075ec0700d3
:10559400f08757000e0a90000442780044479800b0
:1055a4001e0a900004427800544798002e0a900086
:1055b40004427800644798007e0290000442780018
:1055c400344798006e029000044278002447980003
:1055d4005e02900004427800144798004e02900046
:1055e40004427800044f78000042eb0074479800ae
:1055f4000e007800ddf9070000027800e00f520089
:1056040004003a00c14f29003000200082fd070049
:105614000300370051512900300020007efd0700af
:105624000002eb00040078000080fa00000006008d
:105634000200fa00000f78009e007800100020009d
:1056440075fd0700814829001000200072fd070045
:105654000002eb00040078000080fa00000006005d
:105664000200fa00000f78009e007800200020005d
:1056740069fd0700814829002000200066fd07001d
:105684000002eb00040078000080fa00000006002d
:105694000400fa00100798001e009000f9eb0700c0
:1056a40000027800040f78008000eb001e007800f0
:1056b400c4f607000002eb00040078000080fa0042
:1056c400000006000600fa00200798002e00900053
:1056d400eceb070000027800040f78001e02e900da
:1056e4000400780020f907000002780014079800ed
:1056f4001e027800e00f52001a0034001e027800e7
:10570400e40f520017003c001e029000e10f52000b
:105714000a003a009e1f7800e4522900841f780092
:1057240060a12000a3ed0700e487570061a12000d9
:105734003000200038fd0700110037009e1f78005c
:10574400f4532900841f780060a1200099ed07001c
:10575400e487570061a12000300020002efd0700df
:1057640007003700020120001155290060a1200024
:10577400e3eb070061a120003000200026fd0700b4
:105784000002eb00040078000080fa00000006002c
:105794000600fa00200798002e009000b9eb0700dd
:1057a40000027800140798000002eb00040f780050
:1057b4001e029000e00f5200380034001e029000d8
:1057c400e40f520035003c001e029000e40f52002a
:1057d40019003a008000eb001e00900079f60700e3
:1057e4000002eb00040f7800010037001e0fe800f0
:1057f40004fa20009e027800848f5200fbff3400dc
:10580400110020001e0090006ef607001e0290009a
:10581400841f780014562900841f780060a120009a
:1058240064ed0700e487570061a1200030002000e8
:10583400f9fc070020003700110020001e00900032
:1058440060f607000002eb00040f78000100370047
:105854001e0fe80004fa20009e027800848f520094
:10586400fbff34008000eb001e00900055f607009b
:105874001e029000841f780014562900841f7800ab
:1058840060a120004bed0700e487570061a12000d0
:1058940030002000e0fc0700070037000201200070
:1058a4001155290060a1200095eb070061a120009b
:1058b40030002000d8fc07000002eb000400780050
:1058c4000080fa00000006000600fa002007980095
:1058d4002e0090006beb070000027800140798007c
:1058e4000002eb00040f78001e029000e00f52004b
:1058f400400034001e029000e40f52003d003c00c2
:105904001e029000e40f52001d003a001e02900097
:10591400640242008000eb000400780029f60700ce
:105924000002eb00040f7800010037001e0fe800ae
:1059340004fa20009e027800848f5200fbff34009a
:105944001e0290006402420011002000040078004e
:105954001cf607001e029000841f7800745729006b
:10596400841f780060a1200012ed0700e48757002f
:1059740061a1200030002000a7fc070024003700ac
:105984001e0290006402420011002000040078000e
:105994000cf607000002eb00040f7800010037004a
:1059a4001e0fe80004fa20009e027800848f520043
:1059b400fbff34001e029000640242008000eb00f2
:1059c40004007800fff507001e029000841f780091
:1059d40074572900841f780060a12000f5ec0700ab
:1059e400e487570061a12000300020008afc0700f2
:1059f40007003700020120001155290060a1200092
:105a04003feb070061a120003000200082fc07006a
:105a14000002eb00040078000080fa000000060099
:105a24000600fa00200798000002eb00040f78003b
:105a3400050037001e0fe8002e42900084407800d5
:105a4400300020001dfc07000e82e800840078006e
:105a540010002000fbfb070000027800e00f52005a
:105a6400f4ff3a001e027800e00f520003003a00ef
:105a7400e15829003000200067fc07008148290014
:105a84003000200064fc07000002eb0004007800f2
:105a94000080fa00000006000600fa0020079800c3
:105aa4000002eb00040f7800050037001e0fe80029
:105ab4002e4290008440780030002000fffb070055
:105ac4000e82e8008400780020002000ddfb07003f
:105ad40000027800e00f5200f4ff3a001e02780042
:105ae400e00f520003003a00c15a290030002000a0
:105af40049fc0700814829003000200046fc0700cb
:105b04000002eb00040078000080fa0000000600a8
:105b14008a00fa000002eb0014079800153a80008e
:105b2400f40b200004836200640420007505200047
:105b340027742000844b7800854b7800864b7800ce
:105b44002535800004fc2f00048262006401b30048
:105b540024358800a536800004fc2f0004826200ee
:105b64003400b300a43688003535800004fc2f00cf
:105b7400048262007401b30034358800c5368000a5
:105b8400f40f2c008482620004502000048272000e
:105b9400c436880015358000f40f2c00848262001e
:105ba4000480210004827200143588005536800078
:105bb400f40f2c008482620004c02100048272006d
:105bc40054368800153a80000404200004837200cf
:105bd400640420007505200027742000844b78009d
:105be400854b7800864b780005f5070001fb07001c
:105bf40046f807007c030700c3000700660247005d
:105c0400856a2900851f7800156b2900851f780097
:105c1400d56b2900851f78000400780065ec070027
:105c2400e6875700660247008400780030002000b1
:105c3400f9fb0700916f290010002000f6fb070014
:105c44009171290020002000f3fb07006407200065
:105c54000e02420004007800ca0007006407200016
:105c64000e0242000400780013010700040820001b
:105c74000e02420004007800c2000700040820005d
:105c84000e024200040078000b01070001003700f7
:105c9400000000009e029000f47c2000848f5200db
:105ca40003003c0011002000b001200045f507006e
:105cb4009e029000f47c2000848f52000300340084
:105cc4008000eb00b00120003ef507009e0290002a
:105cd40004fa2000848f5200020034000002eb001a
:105ce400140798001e0290000402e80014079800ac
:105cf40066024700040078003300070000027800c1
:105d0400e00f520003003a0034002000040f780032
:105d140013003700660247009173290004007800dd
:105d2400b901070000027800240798002e029000b1
:105d340014427800e04f520003003a00240020008f
:105d4400040f78000600370042002000e1762900a5
:105d54002e0090000202070000027800040f780071
:105d64001e027800e30f5200c9ff32001e027800c1
:105d7400e00f5200100032001e027800e20f5200c1
:105d84000d003200640520000e0242009e1f7800c0
:105d9400c5732900851f78000400780005ec07000e
:105da400e4875700640520000e0242008400780056
:105db4003000200098fb0700717429003000200097
:105dc40095fb0700b3ff37000800fa00300798007e
:105dd4000002eb00040f780064024700840078009e
:105de4003000200017fb070000027800e00f52008b
:105df400410032004e429000844078003000200080
:105e04002efb07004e429000ed4f520003003a0073
:105e1400a1c0b3003000200028fb07004e429000d0
:105e2400ed4f5200190032004e429000e84f5200ec
:105e34000c00320035558000f4042000848f520099
:105e440008003c00355580004e42900086aa200090
:105e540006834200044b78000502e80034558800ac
:105e64000600370034558000e00f52000300340070
:105e7400345580000402e90034558800be029000c5
:105e84000042eb00844a78001b0037001400200015
:105e9400040f78003555800084aa200084824200d3
:105ea4000042eb00844a78000002eb0014079800db
:105eb4000b0037001e029000be0290008482420054
:105ec4001e03900084aa20000402430014427800b8
:105ed400844a78001e0290000402e8001407980027
:105ee400345580009e029000848f5200f1ff3400ec
:105ef4000002eb00345588001e027800040078008c
:105f04000080fa00000006000000fa000002eb0026
:105f1400840888000002eb0034088800f47f240021
:105f24006408880084e0a90094e0a80011e1a800b6
:105f34000080fa00000006000000fa00c300070019
:105f44000080fa00000006000200fa00000f78004a
:105f54001e02780014027800040078000080fa0021
:105f6400000006000200fa00000f78001e0078000e
:105f7400680007001e007800020007000080fa0095
:105f8400000006000200fa00000f78001e037800eb
:105f94006022b8003403980045039800a400070069
:105fa4000002be001e037800140398002503980025
:105fb4000080fa00000006000600fa00200798009e
:105fc4009b0007000002be00048fbe002e0290005a
:105fd40014027800e00f5200230032002e029000d9
:105fe400a402900014029000be0f5200ae8f5a001b
:105ff4000f0036002e02900034039000c40390007a
:106004002e029000a4029000140290003e0142006f
:10601400ae814a000202be000602420087824a00a4
:106024002e03900034039800450398000e003700b7
:106034002e02900034039000c40390002e029000be
:10604400a4029000140290003e011200ae811a00d6
:106054000202be000602420087824a002e0390001c
:1060640034039800450398002e0290001e03be00de
:1060740016029800270298002e029000c402900095
:10608400340290006a2bb900060378006020b9003e
:10609400800378000703430084027800a4002000f2
:1060a400042ab80005034300860278000400be00f9
:1060b4000080fa00000006000200fa00000f7800d9
:1060c4001e007800bcff07001e02780015002000a7
:1060d400050a78001e027800c40290003402900081
:1060e4006a2bb900060378006020b90080037800a9
:1060f4000703430084027800a4002000042ab800a7
:1061040005034300860278000400be000080fa0004
:10611400000006000200fa00000f78001e0078005c
:10612400a5ff07001e0278008002eb00050a780034
:106134001e027800c4029000340290006a2bb90059
:10614400060378006020b900800378000703430049
:1061540084027800a4002000042ab8000503430048
:10616400860278000400be000080fa0000000600e9
:106174000600fa00200798002d0007000003be0067
:106184002e02900005002000041f430005974b00d9
:1061940000000000260007000002be00be0f5200ef
:1061a400ae8f5a00fbff39000080fa0000000600a1
:1061b4000600fa00200798001d0007000002be0038
:1061c400048fbe002e029000e90f52000c0036002e
:1061d400ae029000a4002000809fbe0011000900c0
:1061e4008482d80000027800810278004f00be004b
:1061f400050020001e0f42005e974a00050037008c
:1062040014002000050020001e0f42005e974a0083
:1062140000000000060007000002be00be0f52008e
:10622400ae8f5a00fbff39000080fa000000060020
:106234000000fa0005000700d4578000e5578000ed
:106244000400be000080fa00000006000200fa000c
:10625400c6578000d4578000e557800004027800b8
:10626400040f53001e0278006123b800d457800045
:10627400e55780000602420087824a00d45788000e
:10628400e55788000080fa0000000600841f7800ab
:106294000000fa000002eb0034088800c4578000b4
:1062a4000402e800c457880084e0a9000080fa00d2
:1062b4004f027800004006000600fa00881f7800ac
:1062c40010079800210798000002eb00040f7800e3
:1062d4001e02900014427800e04f520002003a007f
:1062e4000002eb00440037001e027800ae0290006a
:1062f40004824200144278000402fb000400780087
:10630400d9e80700000478001e0278009e0290007d
:1063140004824200144278000402fb000400780066
:10632400d1e8070000027800840f54001400320002
:106334002e0290000402e800240798002e02900028
:1063440014427800e04f520002003a000002eb00d1
:10635400290037002e02900094427800c4c7b3008d
:1063640084cf5200f2ff3a002e0290000402e800ab
:10637400240798000002eb00040f7800190037008e
:106384001e0fe8001e027800ae0290000482420054
:1063940014427800e04f5200070032001e027800d9
:1063a400ae0290000482420094427800c4c7b30055
:1063b40084cf52000b003a001e0278009e02900027
:1063c400048242001442780004407800520007001e
:1063d40000027800e00f520002003a001e0278002a
:1063e40005003700740220009e027800848f52005a
:1063f400bdff34001e027800040078004f047800ca
:106404000080fa00000006000600fa001007980059
:10641400210798000082eb00040f78000d0037007c
:106424001e029000944278001e0278002e03900011
:10643400040243001442780084cf520005003a005d
:106444001e0290000402e800140798000082eb008a
:10645400040f78001e0fe8001e027800ae029000c0
:106464000482420014427800e04f5200ecff3a00ec
:106474001e029000040078000080fa00000006006c
:106484000200fa00000f7800217f29001e00780026
:10649400ddff070000027800040f78001e02780078
:1064a40094427800d4c2b30084cf52000500320075
:1064b4001e02780094427800b4c2b30084cf520024
:1064c40001003a001e0fe800517f29001e007800e9
:1064d400cdff070000027800040f7800717f2900c7
:1064e4001e007800c8ff070000027800040f78003f
:1064f4001e02780014427800e04f5200020032007d
:106504000002eb00010037001400200004007800b2
:106514000080fa00000006000200fa00004f780034
:106524001e02fb000400780022e807000002780045
:10653400e00f520004003a00f4c5b3009e42780014
:1065440084cf520002003a001400200001003700fa
:106554000002eb00040078000080fa00000006004e
:106564000a00fa00200798003107980042079800b3
:106574000002eb00040f7800217f29002e00900018
:10658400a1ff070000027800240798001f003700cd
:106594001e0278004222dd00be0290000482420006
:1065a40014027800840078002e00900042ff070057
:1065b40000027800140798001e029000e00f5200b9
:1065c400110032001e029000ae02900004824200cc
:1065d400217f2900040078008bff07000002780067
:1065e400240798001e0278004222dd00be029000bb
:1065f40004824200140290002e0090000400010066
:10660400000278000a0037001e0fe8001e0278001e
:106614004222dd00be02900004824200140278008f
:1066240014427800e04f5200d9ff3a004e02900025
:0c663400040078000080fa00000006005e
:020000040000fa
:10664000160a00009000000000000000fe0a000092
:106650000200000000000000a60a00005200000036
:1066600000000000000b000002000000000000001d
:10667000000800001602000000000000f80a0000f8
:106680000600000000000000f80b000002000000ff
:1066900000000000a20b00002a0000000200000021
:1066a000303132003334350036373800394142005a
:1066b0004344450046003000313233003435360063
:1066c00037383900616263006465660000286e0037
:1066d000756c6c0029000000020b0000a000000097
:1066e00002000000010000000000000000000a009d
:1066f0000000000000000000006400000000000036
:1067000000000000e803000000000000000010008e
:10671000270000000000000000a08600010000002b
:106720000000000040420f00000000000000800058
:1067300096980000000000000000e100f505000050
:106740000000000000ca9a003b00000000000000aa
:10675000e40b5400020000000000e8007648170037
:10676000000000000010a500d4e8000000000000b8
:10677000a0724e0018090000000040007a10f300db
:106780005a0000000080c600a47e8d0003000000b7
:1067900000c16f00f2862300000000008a5d7800cf
:1067a0004563010000006400a7b3b600e00d0000df
:1067b00000e889000423c7008a000000f20b0000f3
:1067c0000600000000000000cc0b000026000000c6
:1067d00002000000f30b000000f30b0009000000b2
:1067e00000020000f50b000000f50b000e02010096
:1067f000000000000000000000000000060202008f
:1068000000000000cc0b0000fa0b000002000000aa
:0c68100002000000010000000000000079
:020000040000fa
:10681c000400fa00004f7800110798001e00900049
:10682c004200070000027800e00f52000200320024
:10683c000002eb000f0037001e029000940278005b
:10684c001e02900014029000048242001e4a78003e
:10685c001e029000140290008402e8001e029000b8
:10686c0034029000848262001e029000150298008f
:10687c0014002000040078000080fa0000000600dc
:10688c000400fa00000f7800110798001e00900019
:10689c003800070000027800e00f520005003200bb
:1068ac009e0278000042eb00844a78000002eb0064
:1068bc00110037001e029000940278001e02900016
:1068cc002402900004824200144278009e02780058
:1068dc00844a78001e029000240290008402e80092
:1068ec001e02900034029000848262001e0290000e
:1068fc002502980014002000040078000080fa00a3
:10690c00000006000200fa00000f78001e0278005a
:10691c008002eb00250298001e0278008002eb003a
:10692c00150298000080fa00000006000200fa0030
:10693c00000f78001e027800140290008402e80018
:10694c001e02780034029000848262001e027800dd
:10695c0024029000848f520002003a0014002000a0
:10696c00010037000002eb00040078000080fa0000
:10697c00000006000200fa00000f78001e027800ea
:10698c00a40290001e02780014029000848f520022
:10699c0002003a0014002000010037000002eb0056
:1069ac00040078000080fa00000006000200fa00e3
:1069bc00000f78001e027800940290001e027800ee
:1069cc0024029000848252001e027800340290004f
:1069dc0004826200040078000080fa0000000600c7
:1069ec000000fa004382a9004362a9004342a900b7
:1069fc004322a9004302a80042e2a80042c2a90017
:106a0c0042a2a800141280000420a1000430a100ae
:106a1c000440a10014128800141280000400a0008d
:106a2c000410a0001412880045e2a90045c2a90078
:106a3c0045a2a9004422a9004402a90041e2a800f1
:106a4c00811f7800821f7800831f7800217420003a
:106a5c006204200073052000824878008348780087
:106a6c0042c7a900cf0178004f017800cf00780011
:106a7c004535800004fc2f00048262003401b30011
:106a8c0044358800d5368000f40f2c0084826200d7
:106a9c000480200004827200d4368800d536800031
:106aac0004fc2f00048262005400b300d43688002a
:106abc00811f7800821f7800831f780021742000ca
:106acc006204200073052000824878008348780017
:106adc0042c7a800cf0178004f017800cf007800a2
:106aec000080fa00000006000200fa00000f780097
:106afc001e0278004412880000000000041280007e
:106b0c0061026200e00f5200fcff32000002eb0059
:106b1c00040f780044128000040078000080fa0012
:106b2c00000006000000fa0004588000e00f52003c
:106b3c0001003a00ff3ffc00045880000402e8000a
:106b4c00045888000080fa00000006000000fa00db
:106b5c00045880000402e90004588800045880009e
:106b6c00e00f520001003a000000fc000080fa0027
:046b7c00000006000f
:020000040000fa
:020000040005f5
:0457f400023e000071
:020000040000fa
:020000040005f5
:0457f800bdfa0000f6
:020000040000fa
:020000040005f5
:0457fc007f3f0000eb
:00000001FF
